:020000040800F2
:10000000F81A002001010008C1130008B50E00080D
:10001000BD130008A10500081D170008000000001E
:10002000000000000000000000000000C9150008EA
:10003000A505000800000000C9140008CD1500083F
:100040001B0100081B0100081B0100081B01000820
:100050001B0100081B0100081B0100081B01000810
:100060001B0100081B0100081B0100081B01000800
:100070001B0100081B0100081B0100081B010008F0
:100080001B0100081B0100081B0100081B010008E0
:100090001B0100081B0100081B0100081B010008D0
:1000A0001B0100081B0100081B0100081B010008C0
:1000B0001B0100081B0100081B0100081B010008B0
:1000C0001B0100081B0100081B0100081B010008A0
:1000D0001B010008FD1600081B0100081B01000899
:1000E0001B0100081B0100081B010008DFF80CD0F1
:1000F00000F01EFA00480047211D0008F81A0020F1
:100100000648804706480047FEE7FEE7FEE7FEE7B1
:10011000FEE7FEE7FEE7FEE7FEE7FEE7DD16000886
:10012000ED000008202A04DB203A21FA02F0002129
:10013000704721FA02F3D040C2F1200291400843F7
:100140001946704740EA01039B0703D009E008C93C
:10015000121F08C0042AFAD203E011F8013B00F88C
:10016000013B521EF9D27047D2B201E000F8012BD8
:10017000491EFBD270470022F6E710B513460A4627
:1001800004461946FFF7F0FF204610BD421C10F848
:10019000011B0029FBD1801A704730B480EA0102AC
:1001A00002F0004530F0004221F0004013D090B141
:1001B000C30DD40DC2F31601C0F31600E41A41F4C6
:1001C000000140F400027D34914201D3641C00E040
:1001D0004900002C02DA30BC002070474FF40000C8
:1001E0000023914201D3891A034340084FEA410199
:1001F000F7D151B1914202D14FF0004105E002D256
:100200004FF0010101E06FF0010103EBC4502844FD
:1002100030BC00F0F9B82DE9FE4F804681EA0300BA
:10022000C00F0C46009021F0004123F00045B8EBD0
:100230000200A94105D24046214690461C460B4685
:10024000024623F00040104347D0270DC7F30A00B1
:10025000C3F30A510290401A019040286BDAC3F3AD
:10026000130040F4801B0098924620B10023D2EB8B
:10027000030A63EB0B0B01985946C0F1400250464C
:1002800000F0A1F806460D4650465946019A00F086
:10029000A9F810EB08006141002487EA115284EAB2
:1002A000E7731A4340D0009A62B3019A012A4FEAD9
:1002B000075215DC001B61EB02014FF0004202EA1D
:1002C0000752CDE90042001C41F5801132462B4611
:1002D00000F0E0F803B0BDE8F08F40462146F9E7B2
:1002E000001B61EB0201001C41F5801300185B410B
:1002F0002018A2F5001747EB030140EAD570B619A4
:100300006D4111E06D084FEA360645EAC0754FEAC7
:100310000752001B61EB0201001C41F580114908E6
:100320004FEA30000019514132462B4603B0BDE878
:10033000F04F00F0A0B80098012240000023D0EB5D
:10034000020263EBE073009821464FEAE074B8EBD9
:10035000000061EB0401E9E783F000435BE781F013
:10036000004158E796230022114600F056B8C1F329
:100370000A5210B5C1F3130140F2FF3341F480116A
:100380009A4201DA002010BD40F233439A42A2F2B1
:10039000334203DC5242FFF7C5FE10BD904010BD52
:1003A00000F0004230F000400AD0C10D01F560714C
:1003B000C0F3160042EA0151C208400711437047DA
:1003C000002001467047202A04DB203A00FA02F19F
:1003D000002070479140C2F1200320FA03F3194333
:1003E00090407047202A06DBCB17203A41FA02F0F2
:1003F00043EAE07306E041FA02F3D040C2F1200282
:1004000091400843194670470029A8BF7047401C17
:10041000490008BF20F00100704710B4B0FA80FC1A
:1004200000FA0CF050EA010404BF10BC704749B157
:10043000CCF1200421FA04F411FA0CF118BF0121C7
:1004400021430843A3EB0C01CB1D4FEA00614FEAA7
:10045000102042BF002010BC704700EBC350104476
:100460000029A4BF10BC7047401C490008BF20F001
:10047000010010BC704710B5141E73F1000408DAB7
:10048000401C41F1000192185B411A4301D120F058
:10049000010010BD2DE9F04D92469B4611B1B1FA15
:1004A00081F202E0B0FA80F220329046FFF78BFF33
:1004B00004460F4640EA0A0041EA0B0153465A46F9
:1004C000084313D0114653EA010019D0C8F1400285
:1004D0005046FFF727FE05460E465046594642460F
:1004E000FFF771FF084305D0012004E0204639469C
:1004F000BDE8F08D0020054346EAE0762C43374303
:100500000A986305E40AA0EB08000022FD0A44EA09
:1005100047540A3002D500200146E9E701051019C9
:100520006941DDE9084500196941BDE8F04DA2E7E0
:10053000064C074D06E0E06840F0010394E8070030
:1005400098471034AC42F6D3FFF7D4FD981E00084C
:10055000B81E000810B500F081FF0348816A884783
:1005600002494868804710BD58000020E400002080
:1005700010B50A22084801880848008800F022FFC8
:10058000012805D1044800880449088001F0B4F826
:1005900001F0A6F810BD0000100000201A00002095
:1005A00000BFFEE7704772B600BFFEE70021074AB2
:1005B000D1610749096941F00401054A11611146F9
:1005C000096941F04001116170470000F800002006
:1005D000002002400021074AD1610749096941F022
:1005E0000201054A116111464861096941F0400163
:1005F00011617047F8000020002002400022054BE6
:10060000DA61054A126942F00102034B1A61018066
:1006100070470000F80000200020024000201E4922
:10062000C96801F0100139B11C49C96941F00201E2
:100630001A4AD16140F010001749C96801F004015D
:1006400039B11649C96941F00101144AD16140F03C
:1006500004001149C96901F0010169B10F49C96973
:1006600041F004010D4AD16100BF0B49C96921F075
:100670000101094AD16100BF00BF40F20111884267
:1006800006D10549C96921F00101034AD16101E0A0
:100690000149C86000BF704700200240F8000020F8
:1006A00070B5044600F09CFA054609E0601C38B1BC
:1006B00024B100F095FA401BA04201D9032070BD7F
:1006C0001248C06800F001000028EFD10F48C06850
:1006D00000F0200020B100BF20200C49C86000BFFE
:1006E0000A48C06800F0100048B90848C06900F026
:1006F000010020B90548C06800F0040018B1FFF7F8
:100700008DFF0120DBE70020D9E700000020024038
:100710002DE9F04104460E460127002500BF26487A
:10072000007E012802D10220BDE8F081012022498B
:10073000087600BF2068022813D14CF25030FFF732
:10074000AFFF90BB0120FFF731FF4CF25030FFF7B5
:10075000A7FF07461948006920F0040017490861FF
:1007600023E04CF25030FFF79BFFF0B94FF0FF3021
:100770003060A56812E02846FFF72CFF4CF250309D
:10078000FFF78EFF07460D48006920F002000B4975
:1007900008610FB1356007E005F58065D4E9021006
:1007A00001EB8020A842E6D800BF00BF002002492C
:1007B000087600BF3846B7E7F80000200020024066
:1007C0000348006940F0800001490861002070473B
:1007D000002002402DE9FE4F05468B4617469846FD
:1007E000012600240020029000BF2448007E01283A
:1007F00002D10220BDE8FE8F01202049087600BF0B
:100800004CF25030FFF74CFF064686BB012D02D15B
:100810000120029006E0022D02D10220029001E0A8
:100820000420029000241EE02201B946C246484638
:100830005146FFF777FC80B20190022000FB04B024
:1008400000900199FFF7DAFE4CF25030FFF728FFD5
:1008500006460B48006920F001000949086106B10D
:1008600004E0601CC4B202988442DDDB00BF00BF1C
:1008700000200249087600BF3046BBE7F8000020A0
:100880000020024000200849096901F0800151B1AF
:100890000649054A5160064951601146096901F04F
:1008A000800101B10120704700200240230167450B
:1008B000AB89EFCD2DE9F8470346002294466EE15F
:1008C0004FF0010808FA02F4D1F8008008EA0400A9
:1008D000A0427DD1DFF8DCA2D1F80480A8EB0A09A0
:1008E000D0453AD014DCB8F1030F50D009DCB8F190
:1008F000000F31D0B8F1010F1CD0B8F1020F49D16F
:1009000020E0B8F1110F18D0B8F1120F42D11EE05B
:10091000B9F5881F25D006DCB9F5803F20D0B9F5A0
:10092000801F37D11AE0B9F5001F18D0B9F5041FA0
:1009300030D117E0D1F80CC02DE0D1F80C8008F1CF
:10094000040C28E0D1F80C8008F1080C23E0D1F861
:100950000C8008F10C0C1EE000BF00BF00BF00BF00
:1009600000BF00BFD1F80880B8F1000F02D14FF0EE
:10097000040C0BE0D1F80880B8F1010F03D14FF05F
:10098000080C1C6102E04FF0080C5C6103E04FF0C2
:10099000000C00E000BF00BFFF2801D8984601E02E
:1009A00003F104084646FF2802D84FEA820803E014
:1009B000A2F108084FEA88084746D6F800804FF0B1
:1009C0000F0909FA07F928EA09080CFA07F900E003
:1009D00088E048EA0908C6F80080D1F8048008F0E9
:1009E0008058B8F1805F7DD100BFDFF8CC81D8F8A6
:1009F000188048F00108DFF8C091C9F81880C8468F
:100A0000D8F8188008F00108CDF8008000BF00BFBA
:100A10004FEAB9384FEA920958F829504FEA8278DC
:100A20004FEA18794FF00F0808FA09F825EA080587
:100A3000DFF88881434502D14FF0000816E0DFF867
:100A40008081434502D14FF001080FE0DFF8748147
:100A5000434502D14FF0020808E0DFF86C814345BE
:100A600002D14FF0030801E04FF004084FEA827909
:100A70004FEA197908FA09F848EA0505DFF84C81C8
:100A80004FEA920948F82950D1F8048008F48018F8
:100A9000B8F5801F0AD1DFF83881D8F8008048EA1D
:100AA0000008DFF82C91C9F8008009E0DFF8208108
:100AB000D8F8008028EA0008DFF81491C9F800800F
:100AC000D1F8048008F40018B8F5001F10D1DFF841
:100AD000008108F10408D8F8008048EA0008DFF82F
:100AE000F09000E05AE009F10409C9F800800DE037
:100AF000DFF8DC8008F10408D8F8008028EA000854
:100B0000DFF8CC9009F10409C9F80080D1F804801D
:100B100008F40038B8F5003F0ED1DFF8B480A8F132
:100B20000408D8F8008048EA0008DFF8A490A9F18A
:100B30000409C9F800800DE0DFF89480A8F10408EA
:100B4000D8F8008028EA0008DFF88490A9F10409A9
:100B5000C9F80080D1F8048008F48038B8F5803FE7
:100B60000ED1DFF86C80A8F10808D8F8008048EAB8
:100B70000008DFF85C90A9F10809C9F800800DE0D1
:100B8000DFF84C80A8F10808D8F8008028EA0008AF
:100B9000DFF83C90A9F10809C9F80080521CD1F88F
:100BA000008028FA02F8B8F1000F7FF489AEBDE8A2
:100BB000F8870000000011100010024000080140FA
:100BC000000C0140001001400014014008000140E9
:100BD000080401400AB1016101E00B0403617047A0
:100BE00001480068704700000000002003480068CA
:100BF0000349097808440149086070470000002053
:100C00000800002010B50848006840F010000649B0
:100C10000860032000F098F80F2000F007F800F0BB
:100C20002BF8002010BD00000020024070B50446E3
:100C30000E4800784FF47A71B1FBF0F00C49096866
:100C4000B1FBF0F5284600F01BF908B1012070BD9A
:100C5000102C07D200222146501E00F037F805481C
:100C6000046001E00120F2E70020F0E70800002026
:100C70000C0000200400002008B500BF1148806966
:100C800040F001000F4988610846806900F00100CA
:100C9000009000BF00BF00BF0846C06940F0805010
:100CA000C8610846C06900F08050009000BF00BFD6
:100CB00000BF0549486820F0E06040F000704860DF
:100CC00000BF08BD00100240000001402DE9F05FA8
:100CD00080460D461646002700F022FD074639469D
:100CE0002A46334601F00700C0F1070ABAF1040FA3
:100CF00002D94FF0040A01E0C0F1070AD14600F121
:100D0000040ABAF1070F02D24FF0000A01E0A0F185
:100D1000030AD4464FF0010A0AFA09FAAAF1010AB5
:100D20000AEA020A0AFA0CFA4FF0010B0BFA0CFB62
:100D3000ABF1010B0BEA030B4AEA0B0421464046D8
:100D400000F0F6FCBDE8F09F00BF00F00702064B84
:100D500019684FF6FF031940044B0B4343EA022185
:100D6000014B196000BF70470CED00E00000FA0570
:100D700010B5FFF735FF04463D48006840F001001C
:100D80003B49086006E0FFF72BFF001B022801D952
:100D9000032010BD3648006800F002000028F2D0A1
:100DA0003348006820F0F80040F0800030490860C7
:100DB000FFF716FF044600202D49486008E0FFF7C2
:100DC0000FFF001B41F28831884201D90320E0E780
:100DD0002748406800F00C000028F0D1254826493B
:100DE000086026480068FFF721FF08B10120D0E71E
:100DF000FFF7F6FE04461E48006820F080701C498C
:100E0000086006E0FFF7ECFE001B022801D9032072
:100E1000BFE71748006800F000700028F2D11449BD
:100E20004860FFF7DDFE04461148006820F41020FA
:100E30000F49086006E0FFF7D3FE001B642801D9C4
:100E40000320A6E70A48006800F400300028F2D129
:100E50000748006820F48020054908600846406A79
:100E600040F0807048620020886000BF91E7000079
:100E70000010024000127A000C0000200400002044
:100E800070B504462546681EB0F1807F01D301206D
:100E90000FE0681E4FF0E02148610F214FF0FF3056
:100EA00000F046FC00204FF0E02188610720086137
:100EB000002070BD00BFFEE708B505498969014300
:100EC000034A9161114689690140009100BF08BD44
:100ED000001002402DE9F04102460B461868C0F3AD
:100EE0000F2595FAA5F0B0FA80F480E00120A0402B
:100EF000284000287AD0082C04D240F2011000FAD1
:100F000004F106E0A4F108004FF00116864046F017
:100F10008061586808280ED11869D66826EA11261B
:100F20000F0A97FAA7F7B7FA87F700FA07F73E43D1
:100F3000D66000BF00BF586802EB116691FAA1FCB1
:100F4000BCFA8CFC4FEA8C084FF00F0C0CFA08FC32
:100F5000376827EA0C0791FAA1FCBCFA8CFC4FEA2F
:100F60008C0C00FA0CFC47EA0C07376000BF58688D
:100F7000012802D05868092838D1986802EB116618
:100F800091FAA1FCBCFA8CFC4FEA8C084FF0030CE0
:100F90000CFA08FC376827EA0C0791FAA1FCBCFAA6
:100FA0008CFC4FEA8C0C00FA0CFC47EA0C0737600B
:100FB00000BFD86802EB116691FAA1FCBCFA8CFC68
:100FC0004FEA8C084FF0040C0CFA08FC376827EA4B
:100FD0000C0791FAA1FCBCFA8CFC4FEA8C0C00FACD
:100FE0000CFC47EA0C07376000BF00BF641C25FA01
:100FF00004F000287FF47AAFBDE8F08110B5044614
:1010000000F098FA2060206800F060FA6060606884
:1010100000F06CFAA060606800F07AFAE06010BD41
:1010200001490860704700000C0000202DE9FF41D5
:1010300004460D4601270026204600F046F8002809
:1010400033D1E9686868084329690843E16841F2D7
:101050000C6291430843E060A868216921F4405183
:101060000143216100BF6869616921F44071014356
:10107000616100BF6846FFF7C1FF0E48844201D19D
:10108000039E08E00C48844201D1029E03E00B4815
:10109000844200D1029E46B1286830B10027314613
:1010A00020462A6800F016F800BF384604B0BDE8B4
:1010B000F08100000038014000440040004800403A
:1010C00001460868C0F3401070470146C868C0F385
:1010D0004030704770B501EBC10303EB011394007E
:1010E000B3FBF4F301EBC10404EB01149500B4FB72
:1010F000F5F46425B4FBF5F404EBC40505EB041426
:10110000A3EB8403322404EB03136424B3FBF4F352
:1011100003F0F00301EBC10404EB01149500B4FBF0
:10112000F5F46425B4FBF5F403EB041401EBC103FF
:1011300003EB01139500B3FBF5F301EBC10505EBE0
:1011400001159600B5FBF6F56426B5FBF6F505EB43
:10115000C50606EB0515A3EB8503322505EB031346
:101160006425B3FBF5F303F00F0323449BB28360C4
:1011700070BD000000B585B0002001900290039082
:10118000049000BF3548806940F0200033498861F1
:101190000846806900F02000009000BF00BF00BF3B
:1011A0000846806940F0040088610846806900F0C4
:1011B0000400009000BF00BF00BF0846806940F0F7
:1011C000080088610846806900F00800009000BFB0
:1011D00000BF002241F612012148FFF7FBFC01226B
:1011E00041F203011F48FFF7F5FC00224FF4F071B4
:1011F0001C48FFF7EFFC41F612000190012002901D
:10120000002003900220049001A91548FFF752FB2B
:1012100041F2E3000190012002900020039003209E
:10122000049001A90F48FFF745FB4FF4807001902F
:1012300001200290002003900220049001A9094897
:10124000FFF738FB4FF400700190002002900390EC
:1012500001A90448FFF72EFB05B000BD00100240B5
:1012600000080140000C01402DE9F0418CB01C2128
:1012700005A8FEF780FF14216846FEF77CFF4FF4B7
:101280008040FFF719FE0420FFF716FE4548009046
:1012900009200190032002900020039069464248F3
:1012A000FFF718FE414800900420019069463E482F
:1012B000FFF710FE25213E4B1B68C3F302200024DC
:1012C00025460346C3F1070CBCF1040F02D94FF0C9
:1012D000040C01E0C3F1070C674603F1040CBCF1F8
:1012E000070F02D24FF0000C01E0A3F1030C664699
:1012F0004FF0010C0CFA07FCACF1010C0CEA040CE9
:101300000CFA06FC4FF0010808FA06F8A8F10108EB
:1013100008EA05084CEA080200BF002904DB1007B0
:10132000030E2448435407E01007040E20480C30F5
:1013300001F00F031B1FC45400BF2520002809DB48
:1013400000F01F02012191404209920002F1E022C7
:10135000C2F8001100BF4FF4E13005900020069064
:10136000079008900C20099000200A900B9005A986
:101370001148FFF75BFE00BF0F48006920F4904062
:101380000D4908610846406920F02A00486100BF05
:1013900000BF0846C06840F40050C86000BF0CB0F1
:1013A000BDE8F081020002040008014004000404CA
:1013B0000CED00E000E400E00038014000BFFEE773
:1013C00000BFFEE710B503461446E01882B29A4209
:1013D00005DD914201DA994207DA012010BD914200
:1013E00003DB994201DA0120F8E70020F6E700006C
:1013F000154909880144144A118014490988014497
:10140000124A1180124909880144114A11800F497A
:101410000988B1F57A7F07D300210C4A11800D4964
:101420000988491C0B4A11800949098842F2107247
:10143000914207D30021064A118007490988491CB7
:10144000054A11807047000010000020160000209F
:101450001800002012000020140000200020104975
:101460000880104908801049088010490880084603
:1014700000880F4908800D4800880E4908800B48F5
:1014800000880D490880094800880C4908800748F1
:1014900000880B490880054800880A490880704781
:1014A000160000201800002012000020100000206C
:1014B0001A0000201C0000201E0000202000002038
:1014C000220000202400002070470000014600BFD9
:1014D0000448406800F0F0000009034A125C21FA59
:1014E00002F0704700100240641E0008014600BF71
:1014F0000548406800F4E060044A02EB10200278DE
:1015000021FA02F07047000000100240741E00082B
:10151000014600BF0548406800F46050044A02EBF1
:10152000D020027821FA02F070470000001002403B
:10153000741E000810B5002400BF0B48406800F07E
:101540000C0020B1042804D0082808D103E0074C7F
:1015500007E0064C05E000F00BF8044601E0034C00
:1015600000BF00BF204610BD0010024000127A00EC
:101570000021002200BF1148406800F4803002467C
:101580001AB1B2F5803F0CD101E00D490BE000BF6C
:101590000A484068C0F34040401C0A4BB3FBF0F1DE
:1015A00001E0074900BF00BF00BF0448406800F4E5
:1015B0007010022303EB9040484370470010024034
:1015C00000093D0000127A007047000010B50120AC
:1015D000FFF70EFF03480121826B9047FFF706FBE0
:1015E00010BD00005800002010B5022038490968DD
:1015F00021F007010143364A116000BF00BF00BF60
:101600003348006800F007000228F8D100BF3148D5
:10161000006840F480302F49086000BF00BF00BF61
:101620002C480068C0F340400028F8D04FF48030C8
:101630004FF4E011274A526822F47C1200F4403340
:101640000B431A43234B5A6000BF00BF1846006883
:1016500040F080701946086000BF00BF00BF1D4801
:101660000068C0F340600028F8D00020194949689C
:1016700021F0F0010143174A516000BF10151146D7
:10168000496821F4E0610143516000BF0020114628
:10169000496821F460510143516000BF02201146A6
:1016A000496821F003010143516000BF00BF00BF42
:1016B0000848406800F00C000828F8D10648FFF7F9
:1016C000AFFC0F20FFF7B2FA08B1FEF76CFF10BDB8
:1016D000002002400010024000A24A0470470000AF
:1016E00010B50348016C884702498868804710BDDF
:1016F00058000020E40000207047000010B50548A5
:10170000FFF7DEFC28B100BF024800680248416BC9
:10171000884710BD003801405800002000BFFEE798
:1017200002480068C0F30220704700000CED00E0A2
:1017300010B5002804DB0A07130E054A135406E00F
:101740000A07140E034A00F00F031B1FD45410BDE8
:1017500000E400E018ED00E002E008C8121F08C134
:10176000002AFAD170477047002001E001C1121F22
:10177000002AFBD17047000070B5144C1449206852
:101780000840B0F1005F1FD172B6FFF7F1FA0020F8
:101790004FF0E02108614861886100BF09E04FF027
:1017A000FF320C4941F820200B4941F82020411C10
:1017B000C8B20828F3DB6568206880F3088800BF9A
:1017C00062B6A84700BFFEE770BD00000028000811
:1017D0000000FE2F80E100E080E200E010B586B05E
:1017E000044600200190029004940120059001A974
:1017F00002A8FEF78DFF06B010BD10B50021C16331
:10180000416801B910BD416800BF00BF00BF01F1D0
:101810000C0353E8003F43F0200201F10C0343E8BE
:101820000024002CF3D100BF00BF00BFEAE738B5A9
:10183000044660684168C9B200916946206800F0BA
:10184000D6FA204600F03CF838BD000070B50446DA
:10185000A08C618C884227DA206880892084204609
:1018600000F034F8208CE18B88421DDC208CD8B14C
:10187000208C40F24C41884203DD206800F06BFA76
:1018800012E0002506E0094A5119206800F06BFAC1
:10189000681C85B2208CA842F5DCE06B20B1218C5D
:1018A00022460248E36B984770BD0000B009002053
:1018B00090F82620012A02D1428C0A4442847047C3
:1018C000012180F82610002141847047002180F812
:1018D00026104184704730B50B46002113E000BF4D
:1018E00044682568C5F3C015002DF9D05D5C4468D7
:1018F000656000BF00BF44682568C5F38015002DF2
:10190000F9D04C1CA1B29142E9DB30BD01218174B8
:101910007047000000200349096808700248034925
:10192000C8637047F00000203119000858000020FB
:101930002DE9F74F8AB006460F460020099008901F
:10194000B44800680078022802D10DB0BDE8F08FDD
:1019500030785A2801D1042F00DAF6E7B078717890
:1019600040EA0129381F484502D0032008900BE0C7
:10197000781E81B2304600F065FA8246781E315CEE
:10198000514501D001200890A3490C980860F478D3
:10199000351D072C79D2DFE804F078042D79B2F1F7
:1019A000D10001209B49096808709C48FEF7EEFBB6
:1019B000401C00F0FF08424698499948FEF7C2FBD8
:1019C000C346A5209649C91E08700BF10100487056
:1019D0008C7008464078811C9148C01E00F032FA95
:1019E0008F4AD21E0BF10301505410464078C01CA0
:1019F0000990E1E06878297840EA01200790E878CA
:101A0000A97840EA012B83480068A0F802B0584644
:101A1000FEF7A8FC014605904FF08940FEF7BDFB9C
:101A200006900798FEF79EFC00900699FEF7B5FB1E
:101A30000190FEF7B5FC00227A4BCDE90201FEF7DA
:101A4000EAFBCDE90401FEF792FC80B2079007980B
:101A500000F04AF94FF00008A5207149C91E08702E
:101A600008F1010048708C7008464078811C6C4871
:101A7000C01E00F0E7F96A4AD21E08F10301505473
:101A800010464078C01C099096E092E0687829786A
:101A900040EA0128A9F1030080B207905D48006880
:101AA000408800FB08F00690A81C05905E4A069945
:101AB0008818079A059900F0EFF84FEA282158484E
:101AC000C01EC17080F804804FF0020BA521017088
:101AD0000BF101005249C91E48708C7008464078CD
:101AE000811C4F48C01E00F0ADF94D4AD21E0BF1CB
:101AF0000301505410464078C01C09905CE04FF040
:101B000000080220434909680870A5204449C91EFD
:101B1000087008F1010048708C7008464078811CFC
:101B20003F48C01E00F08EF93D4AD21E08F1030165
:101B3000505410464078C01C09903DE04FF0020818
:101B400028783749C91EC87068780871A5200870C0
:101B500008F1010048708C7008464078811C3048BC
:101B6000C01E00F06FF92E4AD21E08F10301505436
:101B700010464078C01C09901EE0FFE74FF00008B7
:101B8000A5202749C91E087008F1010048708C7013
:101B900008464078811C2248C01E00F053F9204AB4
:101BA000D21E08F10301505410464078C01C099021
:101BB00002E00220089000BF00BF089830B1012861
:101BC0000AD0022809D003281FD107E01448C01EFC
:101BD000099900F02BF819E000BF00BFA5201049BB
:101BE000C91E0870012048708C700898C8700421C4
:101BF0000B48C01E00F026F90949C91E08710521CD
:101C00000748C01E00F012F800E000BF00BF00BF90
:101C10009BE60000F0000020F4000020831E000876
:101C2000D71600200000E03F0028000870B50446E9
:101C30000D460648006838B1044800682A46214627
:101C4000C36A02480068984770BD0000F400002095
:101C500010B50E480068007820B101280FD0022886
:101C600011D10DE04FF47A720948018809480088C3
:101C7000FFF7A8FB012801D1FFF77EFD04E003E098
:101C8000FFF77AFD00E000BF00BF10BDF0000020AC
:101C900010000020E00000202DE9F04180460D46B4
:101CA0001746FEF7EFFD00BF30200E49C86000BFA9
:101CB000002411E0601CB84204DA295D285C41EA86
:101CC000002600E02E5D08EB0401324600230120CF
:101CD000FEF780FDA01C84B2BC42EBDBFEF770FD7A
:101CE000BDE8F0810020024070B50546FEF7CAFD50
:101CF00000BF30200849C86000BF002406E0074943
:101D000001EB8420FFF76AFD601C84B2AC42F6DB75
:101D1000FEF756FD70BD00000020024000280008BC
:101D2000FEF770FFFFF760FCFFF724FAFFF79CFA5D
:101D3000FEF710FC01E0FEF71BFCFCE770B5034664
:101D40000C4603E014F8015B03F8015B151EA2F1D9
:101D50000102F7D170BD00B97047002141610161F6
:101D6000C16000BFF8E770B504460D460CB900200D
:101D700070BDE06808B90020FAE745B1D4E9000673
:101D8000236903FB060132462846FFF7D7FF206987
:101D9000401CA16890FBF1F201FB12002061E06899
:101DA000401EE0600120E3E770B504460D460CB923
:101DB000002070BDD4E90210884201D10020F8E76C
:101DC00045B1D4E90016636903FB06103246294683
:101DD000FFF7B4FF6069401CA16890FBF1F201FBC2
:101DE00012006061E068401CE0600120E1E770B52E
:101DF00004460D460CB9002070BDD4E9021088429B
:101E000004DA29462046FFF7CFFFF5E745B1D4E9CC
:101E10000016636903FB061032462946FFF78EFF62
:101E20006069401CA16890FBF1F201FB1200606147
:101E30002069401CA16890FBF1F201FB12002061B7
:101E40000120D9E710B502460B460024002104E02A
:101E5000505C2044C4B2481C81B29942F8DB604215
:101E6000C0B210BD00000000000000000102030429
:101E7000060708090000000001020304081C3044A2
:101E8000586C8056302E3030312E3000000000006B
:101E90000000000000000000B81E00080000002044
:101EA000F800000058170008B01F0008F8000020D4
:101EB000001A000068170008000000001000000071
:101EC0000100000000127A00000000000000000085
:101ED0000000000000000000000000000000000002
:101EE00018010020010000004C0400000000000068
:101EF0000000000000000000640500200100000058
:101F00004C04000000000000000000000000000081
:101F1000280000200038014000000240000002407C
:101F200005040100FC0D00201C0E002020004C04C4
:101F3000000000000A000000FB170008D718000886
:101F40000D1900082F180008B11800080000000043
:101F50004D180008400000200044004000000240EE
:101F600000000240020101006812002088120020D7
:101F700020004C040000000005000000FB170008D2
:101F8000D71800080D1900082F180008B11800080C
:101F9000000000004D1800080000000000000000D4
:101FA00015190008511C0008E40000200000000082
:04000005080000ED02
:00000001FF
